:100000000C94E5000C9417110C94F0100C94C9108A
:100010000C94A2100C940D010C940D010C947B1007
:100020000C940D010C946C130C94F7190C94691A30
:100030000C940D010C940D010C940D010C940D0108
:100040000C940D010C940D010C940D010C940D01F8
:100050000C940D010C940D010C940D010C943110B5
:100060000C940D010C94D41C0C94AE1C0C940D013A
:100070000C940D010C940D010C940D010C940D01C8
:100080000C940D010C940D010C940D010C940D01B8
:100090000C942E050C940D010C940D010C940D0183
:1000A0000C940D010C9432030C940D010D0D100DE8
:1000B000FF0C030D090D310D310D310D140D180D0F
:1000C0001C0D220D260D310D2C0D0000000024000A
:1000D00027002A002D003000000000002500280025
:1000E0002B002E0031000000000200090F00000369
:1000F0000401000C000000000000000000000000EF
:100100000000000000000000002300260029002C51
:10011000002F000404040404030405020202020484
:100120000302020202060606060606040402020292
:1001300004040408020110408040102040804080E8
:10014000080204018040201002011080102040406D
:1001500020080B0002020201000904000001020253
:1001600000000524001001052401010104240206F9
:100170000524060001070581031000400904010061
:10018000020A000000070502024000000705830282
:100190004000000403090412010002EF0201404183
:1001A00023368000010102030141726475696E6F9C
:1001B000204C4C430041726475696E6F204C656F32
:1001C0006E6172646F005C259A1D11241FBECFEF13
:1001D000DAE0DEBFCDBF12E0A0E0B1E0E2E9F7E592
:1001E00002C005900D92A632B107D9F725E0A6E22C
:1001F000B2E001C01D92A430B207E1F710E0C4EEF6
:10020000D0E004C02197FE010E94A428C33ED1077C
:10021000C9F70E94C91D0C94BC2B0C94000080915E
:100220007502E0917602F0917702882311F08491B3
:1002300001C080819FEB980F9A3110F4805E089581
:10024000803269F42091760230917702A9014F5FE4
:100250005F4F5093770240937602232B01F7089566
:100260001F93CF93DF930E940F01C0E0D0E01AE00C
:1002700090ED980F9A30B8F41C9F90011D9F300D9F
:100280001124E901C80FD11D87FDDA95E09780910F
:10029000760290917702019690937702809376028E
:1002A0000E940F01E5CFCE01DF91CF911F910895FC
:1002B0002F923F924F925F926F927F928F929F9276
:1002C000AF92BF92CF92DF92EF92FF920F931F9364
:1002D000CF93DF93CDB7DEB727970FB6F894DEBF85
:1002E0000FBECDBF9F838E831B014D838091720211
:1002F00081111BC081E080937202109272001092F3
:10030000C00094E09093C10099E09093C200809364
:10031000C30083E08093BF0088EE8093D1001092E9
:10032000BF001092D200579A7894109209012E8142
:100330003F8137FF05C03F773F832E830AE001C02E
:1003400001E088E2089F802D112490E04E815F81BA
:100350004817590708F4C2C0013039F441315742F7
:1003600020F0E0E1F7E2FF83EE83802E912CA12CB8
:10037000B12C8E819F81969587959C0140E050E03D
:1003800029833A834B835C834E815F812A01612CF0
:10039000712CA501940160E072E18AE790E00E946F
:1003A000602829813A814B815C81620F731F841F11
:1003B000951FA30192010E941E2769017A01EE2474
:1003C000FF2410E01F5FC11434E0D306E104F10400
:1003D00008F120E032E14AE750E0012E04C05595D3
:1003E0004795379527950A94D2F7C501B4010E9425
:1003F000602829813A814B815C81620F731F841FC1
:10040000951FA30192010E941E2769017A01EE2423
:10041000FF24D8CF0A3049F48E819F8105966AE087
:1004200070E00E947C287F836E834E815F81483E0E
:1004300083E0580759F09101DA010E94A92728EEBC
:1004400033E040E050E00E941E2719011092720034
:100450008091C100807F182B1093C100BB27AF2D66
:100460009E2D8D2D8093BF00C092D1002D81203113
:1004700008F02FE080E190E0821B910904C0F6941F
:10048000E794D794C7948A95D2F78D2D99278093B6
:10049000BF00C092D200309274022092730289B3DE
:1004A0008FEF89BB84E08093720027960FB6F89493
:1004B000DEBF0FBECDBFDF91CF911F910F91FF9097
:1004C000EF90DF90CF90BF90AF909F908F907F90F4
:1004D0006F905F904F903F902F9008959F838E83F1
:1004E00044CF85ED8093BC008091BC0084FDFCCF9F
:1004F00010920E03089540914A02262F30E0240FF7
:10050000311D21323105DCF420910E032430C9F471
:10051000FC0180E090E0861758F430914A02219166
:10052000DC01A85DBD4FA30FB11D2C930196F3CF45
:1005300080914A02680F60934A0280E0089581E04A
:10054000089582E008950895E091C7028091C6025F
:10055000E81730F4F0E0E853FD4F808190E0089513
:100560008FEF9FEF08959091C7028091C602981770
:1005700050F4E92FF0E0E853FD4F208130E09F5F19
:100580009093C70202C02FEF3FEFC90108958091F9
:10059000C60290E02091C702821B91090895CF9274
:1005A000DF92EF92FF920F931F93CF93DF937C0123
:1005B000262F972F8A0180910F03882391F0C62F51
:1005C000D72F6E01C40ED51ECC15DD0571F06991D3
:1005D000D701ED91FC910190F081E02DC7010995C3
:1005E000F3CF642F822F0E947B02C801DF91CF914D
:1005F0001F910F91FF90EF90DF90CF900895CF93D0
:10060000DF931F92CDB7DEB7698320910F032223BA
:10061000D1F020913103203240F021E030E0FC01A4
:100620003383228380E090E015C080911003E82F8F
:10063000F0E0EF5EFC4F998190838F5F8093100311
:100640008093310305C061E0CE0101960E947B02D8
:1006500081E090E00F90DF91CF910895089580E0C0
:1006600090E008951F920F920FB60F9211246F928F
:100670007F928F929F92AF92BF92CF92DF92EF9232
:10068000FF920F931F932F933F934F935F936F931B
:100690007F938F939F93AF93BF93CF93DF93EF930A
:1006A000FF9380917302909174029C012150310953
:1006B0003093740220937302892B09F0B0C1109219
:1006C000720078948091C100807F84608093C10023
:1006D00083E08093BF0088EE8093D1001092BF002A
:1006E0001092D20081E0809309018091760290916E
:1006F0007702892B09F493C18091710281118FC116
:100700009090080180917002882321F080916F02FF
:1007100081117BC17724739470ECA72E7DE5B72EF1
:10072000EAE06E2EF4E08F2EA0EDCA2EA7E0DA2EBE
:10073000B4E0EB2EF12C04EF11E0CFE0D0E00E940A
:100740000F0120917602309177022F5F3F4F309357
:10075000770220937602853609F45EC07CF58136F7
:1007600009F49EC024F58C3309F452C08E3309F489
:100770004DC0813209F08FC080920801D0920501EE
:10078000C0920401F0920701E09206011093030168
:1007900000930201D0930101C093000110927002F6
:1007A000909008018091020190910301C8CF833697
:1007B00089F10CF478C000E022E077C08D36A9F111
:1007C0006CF4873679F15CF18C3609F064C00E94D4
:1007D000300190930701809306014EC08237D1F11A
:1007E0004CF48F3609F057C00E943001982E809348
:1007F0000801A5CF843789F1863709F04CC00E94E3
:100800003001909301018093000199CF939497CF89
:100810009A9495CF00E01FC000E024E046C000E0BD
:1008200025E043C000E027E040C00E940F018C3665
:1008300019F41092700204C07092700210926F024C
:10084000809176029091770201969093770280933F
:10085000760275CF01E020E028C00E943001BC0183
:10086000C5010E947C28669EC001679E900D1124E0
:1008700090930501809304018091040190910501FA
:1008800060910601709107010E947C28709303011A
:100890006093020154CF1092770210927602BFC08B
:1008A00000E029E002C000E02BE0122F3CE0939E24
:1008B000100D11240E940F01982F977F933259F445
:1008C00080917602909177020196909377028093BF
:1008D00076021F5FEFCF8D3269F48091760290919E
:1008E00077020196909377028093760211500E94CE
:1008F0000F01F1CFC0910201D091030181538830E3
:1009000058F4C0910401D09105010E943001BC014E
:10091000CE010E947C28EB017E01F694E7940E94B0
:100920000F018E3261F480917602909177020196E8
:100930009093770280937602CE0DDF1DEECFFE01FD
:1009400080917002882349F0CE0196958795809317
:100950006F0280916F02E81BF109C0910001D091F4
:100960000101011104C01F3F11F0C11105C040E099
:10097000BF0188EE93E046C0113130F020EF210F27
:10098000203618F02FE501C020E0822F6CE00E9495
:100990007028682F74EF7603A0011124BA01620F4A
:1009A000711D9B016C30710540F4220F331FD9017A
:1009B000A65CBE4F2D913C9102C020E030E0873014
:1009C00081F0082E02C0220F331F0A94E2F7823012
:1009D00028F0C90105966AE070E00CC0C901905882
:1009E0000CC0C90126E0880F991F2A95E1F70296ED
:1009F00065E070E00E947C28CB014C2FC03108F0EC
:100A00004FE0BF010E9458010AC060916F0270E080
:100A100040E088EE93E00E94580110926F02FF912F
:100A2000EF91DF91CF91BF91AF919F918F917F9186
:100A30006F915F914F913F912F911F910F91FF9077
:100A4000EF90DF90CF90BF90AF909F908F907F906E
:100A50006F900F900FBE0F901F9018951F920F92DE
:100A60000FB60F9211242F933F934F935F936F9381
:100A70007F938F939F93AF93BF93EF93FF93809157
:100A8000B900887F803609F49CC068F5883209F483
:100A90005BC090F4803109F454C038F4882309F421
:100AA000F6C0883009F44DC0F6C0883109F44CC056
:100AB000803209F45DC0EFC0803409F468C048F4A6
:100AC000803309F455C0883309F0E5C080930C03E6
:100AD000D8C0803509F44FC0883509F45DC088342A
:100AE00009F0D9C0D6C0883909F4C7C0A8F488373E
:100AF00009F467C038F4883609F463C0803709F414
:100B000060C0C9C0883809F4B8C0803909F45FC032
:100B1000803809F0C0C05BC0803B09F486C038F45F
:100B2000803A09F466C0883A09F47FC0B4C0803CBA
:100B300009F4A7C0883C09F4A4C0883B09F48AC022
:100B4000AAC08091E90210C090910B0380910A0322
:100B5000981770F5E0910B0381E08E0F80930B03E3
:100B6000F0E0E651FD4F80818093BB0085EC86C0AC
:100B700080930C038EC0E0910B0381E08E0F809375
:100B80000B038091BB00F0E0E651FD4F8083909114
:100B90000B0380910A036EC0E0910B0381E08E0F7E
:100BA00080930B038091BB00F0E0E651FD4F808302
:100BB00080910D0381116DC081E08093E80284EA89
:100BC00061C083E080930E0310926E02CFCF8091BC
:100BD0006E02803208F051C0E0916E0281E08E0F0B
:100BE00080936E028091BB00F0E0E25BFD4F80835A
:100BF000BDCF85EC8093BC0010920E0380916E02F5
:100C0000803230F4E0916E02F0E0E25BFD4F108242
:100C100060916E0270E0E0914C02F0914D028EE422
:100C200092E0099510926E0236C084E080930E0324
:100C300010924B0210924A02E0914802F091490250
:100C4000099580914A02811105C081E080934A0292
:100C500010922802E0914B0281E08E0F80934B02AC
:100C6000F0E0E85DFD4F80818093BB0090914B02E6
:100C700080914A02981708F479CF85E88093BC00E8
:100C80000AC085EC8093BC0010920E0304C0109241
:100C90000C030E947102FF91EF91BF91AF919F9160
:100CA0008F917F916F915F914F913F912F910F9015
:100CB0000FBE0F901F901895EF92FF920F931F9306
:100CC000CF93DF930E94D2158091AF040E9441140C
:100CD0008091AC049091AD04039731F46091B40419
:100CE0007091B504606804C06091B2047091B3045F
:100CF0008FE194E00E94FF020E94E4138093AB0412
:100D000066E08091AF040E944B140E942510EB0115
:100D10008091C60290E02091C702821B910906973C
:100D2000ACF48091BE049091BF04892B89F30E949A
:100D300025106C1B7D0B8091BE049091BF0486171B
:100D4000970730F781E08093C00474C08091AC04B1
:100D50009091AD040397F9F48FE194E00E94B302FF
:100D6000182F8FE194E00E94B302E82E8FE194E007
:100D70000E94B302D82F8FE194E00E94B302F82EB4
:100D80008FE194E00E94B302C82F8FE194E00E94AB
:100D9000B302082F39C08FE194E00E94B302E82E1D
:100DA0008FE194E00E94B302182F8091AC049091DF
:100DB000AD04892BA9F48FE194E00E94B302F82ED0
:100DC0008FE194E00E94B302D82F8FE194E00E945B
:100DD000B302082F8FE194E00E94B302C82F14C021
:100DE0008FE194E00E94B302082F8FE194E00E940B
:100DF000B302C82F8FE194E00E94B302F82E8FE176
:100E000094E00E94B302D82F212F30E03E29309386
:100E10009A04209399042D2F30E03F2930939C04AD
:100E200020939B042C2F30E0C901902B90939E04BB
:100E300080939D0480919304909194042091850265
:100E400030918602821B930B20918B0230918C0291
:100E5000AC01421B530B5093A2024093A10290930A
:100E60008C0280938B02DF91CF911F910F91FF90A5
:100E7000EF9008958F929F92AF92BF92CF92DF92A0
:100E8000EF92FF920F931F930E94E214E0908A0466
:100E9000F0908B048091830290918402E81AF90A01
:100EA000F0922702E09226020E94A70E2091810272
:100EB00030918202AB01421B530B9A017093820264
:100EC00060938102D7010E94AA2820E030E040EE22
:100ED00050E00E94B128EDE8AE2EF8E3BF2EACE062
:100EE000CA2EDD24D394E12CF12C00E010E00E9406
:100EF000ED2849015A018091910290919202A091AE
:100F00009302B0919402880D991DAA1DBB1D809378
:100F1000910290939202A0939302B09394029D0148
:100F2000552737FD5095452FA8E6B1E00E943D2793
:100F3000BB2797FDB095AB2F80938D0290938E02C7
:100F4000A0938F02B09390021F910F91FF90EF90AA
:100F5000DF90CF90BF90AF909F908F900895EF92C9
:100F6000FF920F931F93CF93DF93CDB7DEB72897F0
:100F70000FB6F894DEBF0FBECDBF61E0CE01019683
:100F80000E9473178BE7E82E82E0F82E89819A8100
:100F9000F70120813181821B930B98878F83BE01DB
:100FA000695F7F4F89E794E00E943E110BE912E0F0
:100FB000F801918380838B819C81F70122813381A9
:100FC000821B930B98878F83BE01695F7F4F8CE6EE
:100FD00094E00E943E11F801938382838D819E816B
:100FE000F70124813581821B930B98878F83BE0183
:100FF000695F7F4F8FE594E00E943E11F801958371
:10100000848328960FB6F894DEBF0FBECDBFDF9164
:10101000CF911F910F91FF90EF900895CF92DF92A3
:10102000EF92FF920F931F93CF93DF93CDB7DEB76D
:101030002C970FB6F894DEBF0FBECDBF84E10E949F
:10104000E617672B682B692B09F080C186E10E94A7
:10105000E617672B682B692B09F078C184E00E94A2
:10106000E617672B682B692B09F070C110E080919F
:10107000E104181788F4E091DF04F091E00483E0C4
:10108000189FE00DF11D112480818F3118F462E06A
:101090000E943D0E1F5FEBCF8091E2048F3170F410
:1010A00060E00E940D0E61E08091E2040E943D0E1E
:1010B0008091EA049091EB040E949C0E8091E304DD
:1010C0009091E404892B01F58CE0EEE2F1E0DE0181
:1010D000119601900D928A95E1F76CE070E080E046
:1010E00090E00E94DD2A009779F02CE0FE01319615
:1010F000DC0101900D922A95E1F79093E40480932E
:10110000E30486E08093E5042091DF043091E0045D
:1011100080E09091E104891750F4F90193E0899FF0
:10112000E00DF11D1124128211828F5FF2CF10E0C9
:101130008091E504181708F07EC09091E304809137
:10114000E404E92FF82FE10FF11DE10FF11DC0803C
:10115000D1804091E6045091E704B60180E090E030
:101160000E94FA128091E8049091E9040E949C0E7A
:1011700000E08091E1040817E0F483E0089F70012B
:101180001124E091DF04F091E004EE0DFF1D808159
:101190008F3168F40E94E40D892B49F4E091DF045B
:1011A000F091E004EE0DFF1D81818F5F81830F5F61
:1011B000E0CF0E94E0128091EA049091EB040E943B
:1011C0009C0E4091E6045091E704B60181E090E066
:1011D0000E94FA128091E8049091E9040E949C0E0A
:1011E00000E08091E1040817E0F493E0099F7001AA
:1011F0001124E091DF04F091E004EE0DFF1D8081E9
:101200008F3168F40E94E40D892B49F4E091DF04EA
:10121000F091E004EE0DFF1D82818F5F82830F5FEE
:10122000E0CF0E94E0128091EA049091EB040E94CA
:101230009C0E1F5F7DCF84E10E94CE139091E1044C
:10124000891758F4E091DF04F091E00493E0899F5E
:10125000E00DF11D1124818101C080E090E09A83AE
:101260008983BE016F5F7F4F82E594E00E943E114B
:101270008093A40286E10E94CE139091E104891725
:1012800058F4E091DF04F091E00493E0899FE00DD1
:10129000F11D1124818101C080E090E09A8389834F
:1012A000BE016F5F7F4F85E494E00E943E11809302
:1012B000A50286E10E94CE139091E104891758F4AB
:1012C000E091DF04F091E00493E0899FE00DF11DCF
:1012D0001124828101C080E090E09A838983BE015D
:1012E0006F5F7F4F88E394E00E943E118093A602D7
:1012F00084E00E94CE139091E104891758F4E091A4
:10130000DF04F091E00493E0899FE00DF11D1124CA
:10131000828101C080E090E09A838983BE016F5F83
:101320007F4F8BE294E00E943E118093A7022C969F
:101330000FB6F894DEBF0FBECDBFDF91CF911F91E6
:101340000F91FF90EF90DF90CF90089583EB91E0A5
:101350000E94761573CE0E9425102091990230913B
:101360009A02621B730B7093980260939702089520
:10137000882311F0479A01C047983F9A08954F92E9
:101380005F926F927F928F929F92AF92BF92CF9215
:10139000DF92EF92FF92CF93DF930E9425104B01D3
:1013A0005C017B010E942510EB01C819D9098091CD
:1013B0009B0290919C02875991098D359140C8F507
:1013C00081E00E94B80980900A0190900B01A090E2
:1013D0000C01B0900D01A501940160E070E088EC73
:1013E00091E40E94B8270E942A282B013C01A50104
:1013F000940160E070E080ED92E40E94B8270E94C2
:101400002A28DC01CB01B2010E949312C436D10517
:1014100008F050C00E942510EB01CE19DF090E9490
:10142000AF0780919F029091A0028937910574F3D4
:1014300041C080919F029091A002895791098B37FA
:10144000914008F040C081E00E94B80980900A01F4
:1014500090900B01A0900C01B0900D01A50194019A
:1014600060E070E088EC92E40E94B8270E942A288D
:101470002B013C01A501940160E070E080ED91E456
:101480000E94B8270E942A28DC01CB01B2010E94E9
:101490009312C436D10570F40E942510EB01CE19C9
:1014A000DF090E94AF0780919B0290919C028739CF
:1014B00091057CF31092A3020E942510709396026E
:1014C0006093950228C05D98559AC0900A01D0900B
:1014D0000B01E0900C01F0900D01A701960160E076
:1014E00070E088EC92E40E94B8270E942A284B0101
:1014F0005C01A701960160E070E080ED92E40E943B
:10150000B8270E942A28DC01CB01B4010E94931263
:1015100081E08093A302DF91CF91FF90EF90DF9065
:10152000CF90BF90AF909F908F907F906F905F9083
:101530004F90089581E00E94B80981E090E00E94F8
:1015400013180E94AF0780919B0290919C02855FC7
:1015500091408B34944050F420919D0230919E0232
:101560002D52314081E0233F314008F080E020914E
:101570009F023091A002255F31402B34344008F0A7
:1015800032C120919D0230919E022D523140233F65
:10159000314008F028C1882309F495C00E94BF2675
:1015A00022E030E040E050E00E941E27DC01CB0149
:1015B0000196A11DB11D81309105A105B10509F06C
:1015C000BFC16EE670E088E690E00E9493120E9430
:1015D000251070939A02609399020E94AB09809142
:1015E000970290919802883E934048F40E94AB097C
:1015F0006EE670E088E690E00E949312F0CF0E94C1
:10160000AF0780919B0290919C028639910584F4EA
:1016100080919F029091A002883791054CF40E941E
:10162000AF076EE670E088E690E00E949312E9CF83
:1016300010929102109292021092930210929402D0
:1016400010928D0210928E0210928F0210929002D0
:101650000E943A0780918D0290918E02A0918F0294
:10166000B09190028A359105A105B1052CF50E9433
:101670003A070E94AF0780919F029091A00289577C
:1016800091098B37914028F464E670E080E090E0A7
:1016900010C080919B0290919C028759910964E649
:1016A00070E08D35914018F484E390E002C08AE147
:1016B00090E00E949312CECF64E670E088E690E05E
:1016C0000E94931265C00E94BF2622E030E040E0F5
:1016D00050E00E941E27613009F087C069E170E088
:1016E00088E690E00E94931210929102109292026A
:1016F000109293021092940210928D0210928E0218
:1017000010928F02109290020E943A0780918D02EF
:1017100090918E02A0918F02B0919002893D9F4FCF
:10172000AF4FBF4F9CF00E943A070E94AF0769E19C
:1017300070E088E690E00E94931280919B02909165
:101740009C02875991098D35914000F70E943A0714
:101750000E94251070939A026093990280918D02E5
:1017600090918E02A0918F02B09190028C3A9F4F7F
:10177000AF4FBF4F6CF00E94AB090E943A070E9426
:10178000AF078091970290919802893B9B4060F04F
:101790001092A3020E942510709396026093950206
:1017A00080E090E00C94131880919B0290919C0231
:1017B000875991098D35914018F460E070E00EC0B2
:1017C00080919F029091A002895791098B37914097
:1017D00018F462E370E002C069E170E088E690E02E
:1017E0000E949312BBCF81111DC064E670E088E6B1
:1017F00090E00E9493120E94251070939A026093C9
:1018000099020E94AB098091970290919802883EBC
:10181000934008F0BDCF0E94AB090E94AF070E9421
:10182000BF09F1CF0E94BF2622E030E040E050E047
:101830000E941E276130C9F664E670E08AE190E0FC
:101840000E949312109291021092920210929302AF
:101850001092940210928D0210928E0210928F02BA
:10186000109290020E943A0780918D0290918E0210
:10187000A0918F02B09190028897A105B1054CF418
:101880000E943A0764E670E08AE190E00E949312B9
:10189000EBCF0E943A0780918D0290918E02A09129
:1018A0008F02B091900285359105A105B1054CF4E8
:1018B0000E943A0764E670E08AE190E00E94931289
:1018C000EACF64E670E088E690E00E9493120E94FE
:1018D000251070939A02609399020E94AB0980913F
:1018E000970290919802883E934098F40E94AB0929
:1018F0000E94AF0764E670E088E690E00E949312D1
:1019000080919F029091A002895791098B37914055
:1019100030F70E94251070939A02609399020E94FA
:10192000AB098091970290919802883E934008F00D
:101930002FCF0E94AB090E94AF070E94BF09F1CFD1
:10194000823009F4CBCE51CFFC01918D228D892FAD
:1019500090E0805C9F4F821B91098F7399270895B7
:1019600080E090E0892B29F00E94841981110C9469
:1019700000000895CF93DF931F92CDB7DEB7698340
:10198000DC01ED91FC910280F381E02D41E050E01B
:10199000BE016F5F7F4F09950F90DF91CF91089542
:1019A00083E08093E9008091F200882319F08AE3B4
:1019B0008093E8000895FC018485958597FD0BC010
:1019C0009FB7F89482E08093E9008091F2009FBF76
:1019D00090E0019608959FB7F89482E08093E90023
:1019E0008091F2009FBF90E0089590E0FC01319754
:1019F000EF30F105B0F5EA5AFF4F0C94A42880911E
:101A000080008F7703C0809180008F7D809380005D
:101A1000089580918000877FF9CF84B58F7702C0C9
:101A200084B58F7D84BD0895809190008F7707C025
:101A3000809190008F7D03C080919000877F80937C
:101A4000900008958091C0008F7703C08091C000FE
:101A50008F7D8093C00008958091C200877F80931E
:101A6000C200089508952E98269A2D98259A2A98AE
:101A7000229A2998219A80EA8093800081E18093BC
:101A8000810080E991E09093870080938600109216
:101A900089001092880010928B0010928A0008959D
:101AA0004FB141708CB186FB882780F98427209143
:101AB000B8025091B7026091890270918A02982F02
:101AC0009227292F30E0942F9527291B3109260FC3
:101AD000371F30938A02209389022091B702909198
:101AE000B802821729F0491719F091E09093B602D5
:101AF0008093B7024093B80208950E94301D90E091
:101B00000895CF93DF931F92CDB7DEB7FC01848594
:101B1000958597FD05C02FEF3FEF358724870BC0D4
:101B2000CE0101960E94061D019719F4898190E06B
:101B300002C08FEF9FEF0F90DF91CF9108950F9329
:101B40001F93CF93DF931F92CDB7DEB78C01FC01BB
:101B50008485958597FF0EC0CE0101960E94061DD3
:101B6000019719F4298130E002C02FEF3FEFF8010F
:101B700035872487F801848595850F90DF91CF9173
:101B80001F910F910895FC01848DDF01A80FB11DF5
:101B9000A35ABF4F2C91848D90E001968F739927A3
:101BA000848FA689B7892C93A089B1898C91806490
:101BB0008C93938D848D981306C00288F389E02D51
:101BC00080818F7D80830895CF93DF93282F30E02D
:101BD000F901EA51FF4F8491F901EE5CFE4FD49177
:101BE000F901ED5EFE4FC491CC2391F081110E946A
:101BF000F50CEC2FF0E0EE0FFF1FEB5FFE4FA59111
:101C0000B491EC91ED2381E090E021F480E002C0FA
:101C100080E090E0DF91CF9108951F93CF93DF9301
:101C2000282F30E0F901EA51FF4F8491F901EE5C71
:101C3000FE4FD491F901ED5EFE4FC491CC23C9F063
:101C4000162F81110E94F50CEC2FF0E0EE0FFF1F14
:101C5000E852FF4FA591B4918FB7F894111105C0C8
:101C60009C91ED2FE095E92302C0EC91ED2BEC93D4
:101C70008FBFDF91CF911F910895CF93DF9390E0B5
:101C8000FC01EE5CFE4F2491FC01ED5EFE4F849161
:101C9000882361F190E0880F991FFC01E653FF4F04
:101CA000C591D491FC01E852FF4FA591B491611107
:101CB00009C09FB7F8948881209582238883EC918E
:101CC0002E230BC0623061F49FB7F8943881822FC5
:101CD000809583238883EC912E2B2C939FBF06C085
:101CE0008FB7F894E8812E2B28838FBFDF91CF9197
:101CF0000895CF93DF93EC01888581110FC081E0B7
:101D000088878A85882311F062E001C060E08985B8
:101D10000E943D0E8FE090E00197F1F789850E94C7
:101D2000E40D2B8530E041E08217930709F440E091
:101D3000842FDF91CF9108958230910538F0880F7C
:101D4000991F880F991F05970197F1F708953FB7DD
:101D5000F8948091C2029091C302A091C402B09104
:101D6000C50226B5A89B05C02F3F19F00196A11DFD
:101D7000B11D3FBFBA2FA92F982F8827820F911D21
:101D8000A11DB11DBC01CD0142E0660F771F881F68
:101D9000991F4A95D1F708958F929F92AF92BF9263
:101DA000CF92DF92EF92FF926B017C010E94A70E0F
:101DB0004B015C01C114D104E104F104F1F00E9473
:101DC000A70EDC01CB0188199909AA09BB09883E35
:101DD0009340A105B10570F321E0C21AD108E108D2
:101DE000F10888EE880E83E0981EA11CB11CC11476
:101DF000D104E104F10419F7DDCFFF90EF90DF90FB
:101E0000CF90BF90AF909F908F9008958F929F92A8
:101E1000AF92BF92CF92DF92EF92FF920F931F93F8
:101E2000CF93DF935C016B017A01809123018823BA
:101E300009F45BC08091F304882309F456C08091B3
:101E4000790280FF05C08091E00082608093E0000D
:101E5000E70110E00AEF83E0882E9AE3992E20979D
:101E6000D9F10E94301D81110AC0015009F43DC012
:101E700061E070E080E090E00E94CC0EF0CF282F6F
:101E800030E0C217D3070CF48C2F4FB7F894809230
:101E9000E9009091E80095FF1DC0282F30E0C21B9B
:101EA000D30BF601982F915020F081918093F1008F
:101EB000FACFC20ED31E112319F09092E80009C088
:101EC0008091E80085FD06C09092E80011E020971F
:101ED00009F010E04FBFC3CF1111C3CF5D9884E666
:101EE0008093ED041E141F0444F081E090E0F5019E
:101EF0009383828380E090E001C0C701DF91CF919E
:101F00001F910F91FF90EF90DF90CF90BF90AF9017
:101F10009F908F9008957F928F929F92AF92BF92E1
:101F2000CF92DF92EF92FF920F931F93CF93DF93A5
:101F3000FC0122853385232B09F479C07B01EC0158
:101F4000D12C8C85D816F0F40D2D10E08E859F8550
:101F5000F801EE0FFF1FEE0DFF1D91838083EA85D0
:101F6000FB85E00FF11F61E080810E940D0E8A85E4
:101F70009B85FC01E00FF11F61E080810E943D0E16
:101F8000D394DFCF83E290E00197F1F710E08C85E6
:101F90001817A8F4C12ED12CEA85FB85EC0DFD1D88
:101FA00060E080810E943D0E8A859B85FC01EC0DDE
:101FB000FD1D60E080810E940D0E1F5FE8CF0E9432
:101FC000A70E4B015C010E94A70EAB01BC01481992
:101FD00059096A097B098E859F85A0E0B0E0481702
:101FE00059076A077B0718F50E94A70E6B01C818EE
:101FF000D908712C8C85781630F7072D10E0EA850A
:10200000FB85E00FF11F80810E94E40D892B51F4C4
:10201000000F111FF701E00FF11F80819181C81699
:10202000D90610F07394E6CFD182C082FBCFDF9146
:10203000CF911F910F91FF90EF90DF90CF90BF90C5
:10204000AF909F908F907F9008952FB7F8946091F4
:10205000BE027091BF028091C0029091C1022FBF59
:1020600008951F920F920FB60F9211242F933F9352
:102070008F939F93AF93BF938091BE029091BF02C5
:10208000A091C002B091C1023091BD0223E0230FA4
:102090002D3720F40196A11DB11D05C026E8230FA0
:1020A0000296A11DB11D2093BD028093BE029093A4
:1020B000BF02A093C002B093C1028091C20290916E
:1020C000C302A091C402B091C5020196A11DB11D29
:1020D0008093C2029093C302A093C402B093C5023E
:1020E000BF91AF919F918F913F912F910F900FBE14
:1020F0000F901F9018951F920F920FB60F921124F8
:102100002F933F934F935F936F937F938F939F93FF
:10211000AF93BF93EF93FF93E0911601F0911701F6
:102120000995FF91EF91BF91AF919F918F917F9111
:102130006F915F914F913F912F910F900FBE0F9034
:102140001F9018951F920F920FB60F9211242F9384
:102150003F934F935F936F937F938F939F93AF932F
:10216000BF93EF93FF93E0911401F091150109954E
:10217000FF91EF91BF91AF919F918F917F916F915F
:102180005F914F913F912F910F900FBE0F901F9035
:1021900018951F920F920FB60F9211242F933F9311
:1021A0004F935F936F937F938F939F93AF93BF935F
:1021B000EF93FF93E0911201F09113010995FF91C4
:1021C000EF91BF91AF919F918F917F916F915F91AF
:1021D0004F913F912F910F900FBE0F901F90189528
:1021E0001F920F920FB60F9211242F933F934F938C
:1021F0005F936F937F938F939F93AF93BF93EF936F
:10220000FF93E0911001F09111010995FF91EF9179
:10221000BF91AF919F918F917F916F915F914F91FE
:102220003F912F910F900FBE0F901F9018951F9206
:102230000F920FB60F9211242F933F934F935F93FA
:102240006F937F938F939F93AF93BF93EF93FF937E
:10225000E0910E01F0910F010995FF91EF91BF916F
:10226000AF919F918F917F916F915F914F913F912E
:102270002F910F900FBE0F901F901895CF92DF9265
:10228000EF92FF920F931F93CF93DF93FC01208176
:10229000DB018D919C91308552814381A52FB42F14
:1022A000A30FB11DA30FB11D4D915C911197BC01FE
:1022B000641B750BAB01052E000C660B770BC184FC
:1022C000D284E384F4844C0D5D1D6E1D7F1D418717
:1022D0005287638774878D939C938085A681B7818D
:1022E000A80FB11D8C9181110BC021508085A68152
:1022F000B781A80FB11D8C91821708F452C046C057
:1023000010E09FEF980FF2800381A08564817581B2
:10231000492F50E0EB01C40FD51F3881CF2DB02FCE
:10232000D02FCA0FD11DCA0FD11DAF2DA30FB11DC4
:10233000A30FB11D0990D881C02D0D90BC91A02D87
:10234000CA17DB075CF5DB01A80FB11D3C93A48124
:10235000B581A40FB51F8C91A681B781A80FB11DBF
:102360008C918F5F8C93808564817581DB01A40FD4
:10237000B51F8C938085A681B781A80FB11D8C9164
:1023800081508C9311E0892F9111BBCF80858F5F95
:102390008087908189134BC0108649C01111F6CFF8
:1023A000A4CF90E030E08217930784F7F280038196
:1023B000A08564817581AC014F5F5F4FEB01C40F55
:1023C000D51F1881CF2DB02FD02FCA0FD11DCA0F06
:1023D000D11DAF2DA10FB11DA10FB11D0990D88145
:1023E000C02D0D90BC91A02DAC17BD077CF6DB0174
:1023F000A80FB91F1C93A481B581A40FB51F8C91A0
:10240000A681B781A80FB11D8C9181508C938085D6
:10241000A481B581A40FB51F8C938085A681B78157
:10242000A80FB11D8C918F5F8C93CA01BCCF8181A5
:10243000A481B581A80FB11D8C9122819381E22FD7
:10244000F92FE80FF11DE80FF11D80819181DF91D7
:10245000CF911F910F91FF90EF90DF90CF90089553
:10246000CF92DF92EF92FF920F931F93CF93DF9360
:10247000EC018B017A01633071053CF0862F6F3FD0
:10248000710521F01CF08FEF01C083E088836801A3
:10249000D594C794C98262E070E0C8010E94942973
:1024A0009B838A8361E070E0C8010E9494299D8328
:1024B0008C8361E070E0C8010E9494299F838E8321
:1024C000C8860E9DC0010F9D900D1E9D900D11247C
:1024D000092E000CAA0BBB0B89879A87AB87BC8798
:1024E00020E088812817B0F4822F90E0EC81FD81F4
:1024F000E80FF91F2083EE81FF81E80FF91F208389
:10250000880F991FEA81FB81E80FF91FF182E082B1
:102510002F5FE7CFDF91CF911F910F91FF90EF9049
:10252000DF90CF9008950F931F93CF93DF938C018B
:10253000EB018091BC02811105C081E08093BC0257
:102540000E94330D17FF05C011950195110981E017
:1025500001C080E0013991E0190714F000E911E0B1
:1025600010938B0000938A00882311F02A9A01C0EF
:102570002A98229A8091BC02811105C081E0809343
:10258000BC020E94330DD7FF05C0D195C195D1097A
:1025900081E001C080E0C13991E0D90714F0C0E9C1
:1025A000D1E0D0938900C0938800882311F0299A44
:1025B00001C02998219ADF91CF911F910F91089521
:1025C00046983E9AE0E9F0E082E080831092910024
:1025D000109271001082109299001092980010923F
:1025E0009700109296001092950010929400869891
:1025F0008E980895FC01109271009B0146175707B1
:1026000008F49A0146983E9890E8909390001092B2
:102610009100909392003E9AEF2B11F08E9A01C098
:102620008E98869A50939700409396004150510996
:102630005093950040939400309399002093980014
:1026400082E88093900089E1809391000895249816
:102650002C9A6A98729A6E98769A8098889A81E0F5
:102660008093680090E190936B008BBB80E59DE0C8
:102670009093170180931601EAE6F0E080818F7C49
:1026800080618083EE9A8CB182FB882780F98093E9
:10269000BB0293B12091BB0294FB882780F982276B
:1026A0008093BA0210928802109287021092B902A7
:1026B0008FB181708093B8029CB12091B80296FBD3
:1026C000882780F982278093B70210928A0210929D
:1026D00089021092B60208951F920F920FB60F92C0
:1026E00011242F933F934F935F936F937F938F9317
:1026F0009F938CB190E09595879595958795482FF8
:10270000417023B130E054E0359527955A95E1F7B3
:102710008227932781702091BB025091BA02609169
:10272000870270918802982F9227292F30E0942FEA
:102730009527291B3109260F371F309388022093D4
:1027400087022091BA029091BB02821729F04917A3
:1027500019F091E09093B9028093BA024093BB02C2
:102760009F918F917F916F915F914F913F912F91A9
:102770000F900FBE0F901F9018958091DA048F3F35
:1027800061F061E00E943D0E60E08091DA040E94F9
:102790000D0E8BE193E00197F1F708954091E1046C
:1027A0002091DF043091E00490E0941749F02D5F10
:1027B0003F4FF90133975081581721F09F5FF5CFB4
:1027C0008FEF0895892F0895209131039091EC04A3
:1027D000213208F04AC080910E038111FCCF32E013
:1027E00030930E0331E030930D033FEF30930C0331
:1027F00010920B0320930A03A1E1B3E04AEE52E0EA
:10280000FA013E2F341B321718F43D913193F9CF62
:102810001092E9022091E902990F922B9093E9021C
:102820009091E802913061F41092E8029091E902EF
:102830009093BB009091BC0093FDF8CF95EC01C044
:1028400095EE9093BC0090910E039230E1F390913D
:102850000C039F3F79F080910C03803241F080910E
:102860000C03803331F084E005C081E003C082E0D6
:1028700001C083E0109210031092310310920F03F5
:10288000089591E090930F038093EC04109210034D
:1028900010923103089590910E039111FCCF613293
:1028A00008F060E291E090930E0390930D032FEFF8
:1028B00020930C0310920B03260F20930A0390938E
:1028C000E9029091E902880F892B8093E9028091B7
:1028D000E802813061F41092E8028091E90280936D
:1028E000BB008091BC0083FDF8CF85EC01C085EE74
:1028F0008093BC0080910E038130E1F380910B0343
:10290000861710F460910B03AAEEB2E028EC32E0D7
:10291000F9018E2F821B861718F48D918193F9CFC0
:102920001092C7026093C602862F0895CF93C82FD6
:102930000E9441146FE08FE194E00E94FF020E9428
:10294000E41381110FC061E08C2F0E944B14909111
:10295000C6028091C702981729F08FE194E0CF91C9
:102960000C94B3028FEF9FEFCF9108951F93CF93F5
:10297000DF931F92CDB7DEB7182F69830E944114F1
:1029800069818FE194E00E94FF020E94E4138111AB
:1029900012C061E0812F0E944B149091C602809179
:1029A000C702981741F08FE194E00F90DF91CF912B
:1029B0001F910C94B3028FEF9FEF0F90DF91CF9197
:1029C0001F910895BF92CF92DF92EF92FF920F93E3
:1029D0001F93CF93DF9380918F040E94411468EA84
:1029E0008FE194E00E94FF020E94E41366E0809170
:1029F0008F040E944B140E9425107B018091C60217
:102A000090E02091C702821B91090697ACF4809157
:102A1000900490919104892B89F30E9425106E19DE
:102A20007F0980919004909191048617970730F761
:102A300081E08093920433C08FE194E00E94B3025E
:102A4000C82E8FE194E00E94B302B82E8FE194E08B
:102A50000E94B302E82E8FE194E00E94B302D82EC8
:102A60008FE194E00E94B302F82E8FE194E00E947F
:102A7000B3021B2D00E00C291093870400938604F9
:102A8000DD2D20E0C22FCE29D0938904C093880485
:102A9000982F88278F2990938B0480938A04DF9145
:102AA000CF911F910F91FF90EF90DF90CF90BF904B
:102AB00008950F931F93CF93DF93082F162FC6E827
:102AC000D4E089850E944114602F8FE194E00E9438
:102AD000FF02612F8FE194E00E94FF020E94E41345
:102AE0008E83DF91CF911F910F910895CF93DF9344
:102AF000BC018FEC93E00E94991CEC0162E272E051
:102B00008FEC93E00E94991C8C0F9D1FDF91CF9159
:102B100008958BE60E9496148F3F2FEF920781F461
:102B20008AE60E9496148F3F2FEF920761F489E6A0
:102B30000E949614833D910541F521E030E02DC0BF
:102B400021E030E002C020E030E0873D9105D1F087
:102B500081E090E090938E0480938D04019702971A
:102B600038F42130310511F08AE608C08BE606C042
:102B70002130310511F088E601C089E680938F0489
:102B800081E0089582E090E0E5CF88E60E94961407
:102B9000833D910529F420E030E080E090E0DACF39
:102BA00080E00895BF92CF92DF92EF92FF920F9351
:102BB0001F93CF93DF938091AE040E94411468EA83
:102BC0008FE194E00E94FF020E94E4138093AB0423
:102BD00066E08091AE040E944B140E9425107B0198
:102BE0008091C60290E02091C702821B910906974E
:102BF000ACF48091BE049091BF04892B89F30E94AC
:102C000025106E197F098091BE049091BF0486172C
:102C1000970730F781E08093C00433C08FE194E0E0
:102C20000E94B302C82E8FE194E00E94B302B82E36
:102C30008FE194E00E94B302E82E8FE194E00E94BD
:102C4000B302D82E8FE194E00E94B302F82E8FE1F8
:102C500094E00E94B3021B2D00E00C291093940411
:102C600000939304DD2D20E0C22FCE29D09396044B
:102C7000C0939504982F88278F2990939804809368
:102C80009704DF91CF911F910F91FF90EF90DF900C
:102C9000CF90BF9008950F931F93CF93DF93082F8A
:102CA000162FC3E9D4E08C8D0E944114602F8FE170
:102CB00094E00E94FF02612F8FE194E00E94FF02E6
:102CC0000E94E413888FDF91CF911F910F91089597
:102CD0000F931F93CF93DF93082F162FC3E9D4E0F0
:102CE0008B8D0E944114602F8FE194E00E94FF02BF
:102CF000612F8FE194E00E94FF020E94E413888F0D
:102D0000DF91CF911F910F9108952091AC043091E4
:102D1000AD042330310511F0803210F40C944B16C1
:102D20000C9468166FE070E08DE10E94B61489344F
:102D3000910561F06FE070E08EE10E94B614893475
:102D4000910509F0A2C020E030E002C021E030E0AF
:102D500083E090E09093AD048093AC0482309105C1
:102D600039F589E18093AE048EE18093AF0483E06E
:102D700090E09093B3048093B20484E090E0909349
:102D8000B5048093B40487E090E09093B7048093F7
:102D9000B60488E090E09093B9048093B80485E08D
:102DA00090E09093BB048093BA0486E090E030C03A
:102DB0008330910599F1019709F45FC02130310505
:102DC00009F461C088E18093AE048EE18093AF0482
:102DD00083E090E09093B3048093B20484E090E0A9
:102DE0009093B5048093B40485E090E09093B70489
:102DF0008093B60486E090E09093B9048093B80481
:102E000087E090E09093BB048093BA0488E090E060
:102E10009093BD048093BC0481E008952130310576
:102E200011F08EE101C08DE18093AF048093AE0478
:102E300088E090E09093B5048093B40489E090E03A
:102E40009093B3048093B2048AE090E09093B90425
:102E50008093B8048BE090E09093B7048093B6041D
:102E60008CE090E09093BD048093BC048DE090E0F2
:102E70009093BB048093BA04CFCF2130310509F47D
:102E800070CF88E16FCF89E19ECF60E270E089E189
:102E90000E94B614019661F06FE070E08EE10E942E
:102EA000B61421E030E0CC97D9F080E090E052CF2A
:102EB00060E270E088E10E94B614019679F06FE05C
:102EC00070E08EE10E94B61431E020E0CC9709F06A
:102ED00030E0832F922F20E030E03CCF80E0089557
:102EE00082E090E037CFFF920F931F93CF93DF9351
:102EF000CDB7DEB7A0970FB6F894DEBF0FBECDBF3B
:102F00008C01F62E8FEF860F823088F48091DA04E0
:102F10008F3F79F061E00E943D0E61E08091DA041C
:102F20000E940D0E8BE193E00197F1F702C00E9421
:102F3000BD13E091CD04F091CE040190F081E02D1D
:102F4000B8018DEC94E009950E94BD1362E0F61281
:102F500031C0E091CD04F091CE040190F081E02DDC
:102F6000BE016F5F7F4F8DEC94E0099540E080914A
:102F7000D9044817F8F4242F30E0220F331FF8014A
:102F8000E20FF31FA1E0B0E0AC0FBD1FA20FB31F13
:102F90008091DB049091DC042D913C91BC01621B7B
:102FA000730B9B0180819181280F391F318320830E
:102FB0004F5FDDCFA0960FB6F894DEBF0FBECDBF3A
:102FC000DF91CF911F910F91FF9008950F931F9361
:102FD00090E0FC01EE5CFE4F6491FC01ED5EFE4F63
:102FE000E491F0E0EE0FFF1FEB5FFE4F85919491AF
:102FF00008EE13E020E030E040E00E94551D61152E
:1030000071058105910549F0DC01CB010196A11DF7
:10301000B11DBC01CD019F7003C060E070E0CB0129
:103020001F910F9108958F929F92AF92BF92CF926E
:10303000DF92EF92FF920F931F93CF93DF93CDB761
:10304000DEB7A1970FB6F894DEBF0FBECDBF6C01FF
:10305000990FEE08FF08F7FE33C0E0913203F091BC
:1030600033030190F081E02D6DE282E393E0099556
:103070008C0122273327A9012C193D094E095F092C
:1030800019A2CE0181967C019AE0892E912CA12C67
:10309000B12CCA01B901A50194010E948727605D86
:1030A000F70162937F01211531054105510589F72B
:1030B000BF0182E393E00E94991C800F911F1FC003
:1030C000A701960119A28E010F5D1F4F8AE0C82E3D
:1030D000D12CE12CF12CCA01B901A70196010E9463
:1030E0008727605DF80162938F0121153105410545
:1030F000510589F7BF0182E393E00E94991CA196D4
:103100000FB6F894DEBF0FBECDBFDF91CF911F91F8
:103110000F91FF90EF90DF90CF90BF90AF909F9076
:103120008F9008954091F0045091F1042091EE04A5
:103130003091EF0442175307B4F49091E800957072
:10314000E1F39091E80092FD19C08093F100809125
:10315000F0049091F10401968F739927892B19F44B
:103160008EEF8093E8008091F0049091F104019635
:103170009093F1048093F00481E0089580E0089535
:10318000DF92EF92FF920F931F93CF93DF93D82E8E
:103190008A017B01E40EF51EEB01CE15DF0571F00F
:1031A000D7FE03C0FE01849101C088810E9492185D
:1031B00021968111F2CF8FEF9FEF01C0C801DF91FF
:1031C000CF911F910F91FF90EF90DF900895615084
:1031D00030F02091F100FC0120830196F8CF28986F
:1031E00084E68093F2040895CF92DF92EF92FF92EB
:1031F0000F931F93CF93DF936C017A018B01C0E093
:10320000D0E0CE15DF0589F0D8016D918D01D60192
:10321000ED91FC910190F081E02DC6010995892B7B
:1032200011F47E0102C02196ECCFC701DF91CF914E
:103230001F910F91FF90EF90DF90CF900895FC01C8
:10324000538D448D252F30E0842F90E0821B930B0B
:10325000541710F0CF96089501970895FC01918DB1
:10326000828D981761F0828DDF01A80FB11D5D96E8
:103270008C91928D9F5F9F73928F90E008958FEF56
:103280009FEF0895FC01918D828D981731F0828D0A
:10329000E80FF11D858D90E008958FEF9FEF089561
:1032A0000E94A72B0F931F93CF93DF931F92CDB74D
:1032B000DEB782E0898342E450E061E571E080E8B6
:1032C0000E94C0180E94411DDC0112960D911C91B4
:1032D00013970115110569F0D801ED91FC91028059
:1032E000F381E02DBE016F5F7F4FC801099597FF05
:1032F00007C089810F90DF91CF911F910F910895A1
:10330000F80100851185E5CF82E393E00E94A40CCB
:1033100021E0892B09F420E0822F0895EF92FF929B
:103320000F931F93CF93DF93EC0181E0888F9B8DE8
:103330008C8D981305C0E889F989808185FD24C0AA
:10334000F62E0B8D10E00F5F1F4F0F731127E02E2D
:103350008C8DE8120CC00FB607FCFACFE889F9890A
:10336000808185FFF5CFCE010E94C30DF1CF8B8DFB
:10337000FE01E80FF11DE35AFF4FF0820B8FEA893F
:10338000FB898081806207C0EE89FF896083E889BC
:10339000F98980818064808381E090E0DF91CF9122
:1033A0001F910F91FF90EF900895CF93DF93EC0161
:1033B000888D8823C9F0EA89FB89808185FD05C055
:1033C000A889B9898C9186FD0FC00FB607FCF5CF8F
:1033D000808185FFF2CFA889B9898C9185FFEDCFD7
:1033E000CE010E94C30DE7CFDF91CF9108951F92C8
:1033F0000F920FB60F9211248F939F938091E1004B
:103400009091E100937F9093E10083FF0FC01092B1
:10341000E90091E09093EB001092EC0092E390931E
:10342000ED001092F30498E09093F00082FF20C02A
:1034300093E09093E9009091F200992319F09AE3B8
:103440009093E8009091ED04992339F09091ED0468
:1034500091509093ED04992389F19091F20499236E
:1034600039F09091F20491509093F204992341F134
:1034700084FF10C08091E2008E7E81608093E20024
:103480008091E1008F7E8093E100809179028E7EB1
:10349000806111C080FF16C08091E2008E7E806145
:1034A0008093E2008091E1008E7E8093E100809124
:1034B00079028E7E81608093790204C05D9ACDCFBF
:1034C000289AD6CF9F918F910F900FBE0F901F908B
:1034D00018951F920F920FB60F921124CF92DF9280
:1034E000EF92FF920F931F932F933F934F935F930E
:1034F0006F937F938F939F93AF93BF93EF93FF93BC
:10350000CF93DF93CDB7DEB76C97DEBFCDBF109200
:10351000E9008091E80083FFEDC168E0CE014596A7
:103520000E94E71882EF8093E8008D8987FF05C02D
:103530009091E80090FFFCCF03C09EEF9093E800CD
:10354000982F907609F0C6C09E892F89188D911109
:103550000CC0803829F480917A028093F10002C077
:103560001092F1001092F10048C1422F50E0512B0F
:10357000913051F4811141C14130510509F03DC1F3
:1035800080917A028D7F0BC0933061F4811135C137
:103590004130510509F031C180917A0282608093F7
:1035A0007A022BC1953041F48091E80080FFFCCF76
:1035B00020682093E30021C1963009F05FC0EB8CB6
:1035C000FC8C1092E9001092F1041092F004123079
:1035D00091F51092EF041092EE040E94521999E0B6
:1035E000BE016F5F7F4FDB01E92F1D92EA95E9F77E
:1035F00099831A8391E09E8390EA98879AEF99873E
:103600002091F0043091F104275F3F4F3C832B83DE
:103610008D831092E9001092F1041092F004F09260
:10362000EF04E092EE0449E050E080E00E94C01810
:103630000E945219E2C0F092EF04E092EE040E9460
:10364000411DDC011296ED90FC901397E114F104FA
:1036500009F4C0C0D701ED91FC910480F581E02D03
:10366000BE016B5E7F4FC7010995009719F00CF002
:10367000C4C0C7C0F701E084F184E8CF973009F4F3
:10368000C0C0983021F481E08093F100B6C0993039
:1036900009F0B3C0837009F0B4C0EDEAF1E081E055
:1036A00021E036E39081992361F08093E900209333
:1036B000EB0091919093EC003093ED008F5F873099
:1036C00089F78EE78093EA001092EA008F89809351
:1036D000F30493C08B8D9C8D1092E9001092F1043D
:1036E0001092F0049093EF048093EE04898D811181
:1036F00056C08E899D89913A59F4813209F081C072
:1037000047E050E06CE171E080E00E94C01875C0B5
:10371000913209F076C0833289F4888D90E0982F39
:1037200088272F89822BA0E0B0E080931801909326
:103730001901A0931A01B0931B015FC0803269F494
:103740008091E80082FFFCCF67E08CE191E00E946D
:10375000E7188BEF8093E80006C0823209F04DC075
:103760008F898093230180917802882319F0EEEFEE
:10377000FAE002C0E0E0F8E080911C0190911D01A8
:10378000A0911E01B0911F01803B9440A105B1059D
:1037900009F07BC08091230180FF93C076C00E9416
:1037A000411DDC0112960D911C9113970115110515
:1037B00041F1D801ED91FC910190F081E02DBE0125
:1037C0006B5E7F4FC8010995811117C0F801008514
:1037D0001185ECCF113009F44EC0133091F48F896C
:1037E000882309F445C0823081F440E860E185EB2C
:1037F00091E00E943426882321F08EEF8093E80028
:1038000079C081E28093EB0075C0813029F440E8F3
:103810006BE089EA91E0EDCF833099F70E94411D7A
:10382000DC011296ED90FC9013978E010F5F1F4FF5
:103830006801E114F10479F0D701ED91FC91068063
:10384000F781E02DB801C7010995080F111DF70197
:10385000E084F184EECFD8011C92F60101900020A3
:10386000E9F73197BF016C197D0940E0C601C1CF6E
:1038700063E971E002C067E971E06115710509F261
:10388000FB01449150E080E840CF0FB6F894A89532
:1038900080916000886180936000109260000FBE8C
:1038A000A895EE3F2AE0F20739F08091FE0A909148
:1038B000FF0A91838083A1CF1092FF0A1092FE0A23
:1038C0009CCFEE3F8AE0F80731F0808191819093A0
:1038D000FF0A8093FE0A87E797E7918380839BE046
:1038E00088E10FB6F894A895809360000FBE90937E
:1038F000600083CF6C960FB6F894DEBF0FBECDBFCD
:10390000DF91CF91FF91EF91BF91AF919F918F91F7
:103910007F916F915F914F913F912F911F910F91E7
:10392000FF90EF90DF90CF900F900FBE0F901F9001
:1039300018956115710579F0FB0101900020E9F7F8
:103940003197AF01461B570BDC01ED91FC910280D2
:10395000F381E02D099480E090E008951F920F928A
:103960000FB60F9211242F933F934F935F936F9352
:103970007F938F939F93AF93BF93EF93FF9382E3D4
:1039800093E00E94C30DFF91EF91BF91AF919F9182
:103990008F917F916F915F914F913F912F910F90F8
:1039A0000FBE0F901F9018951F920F920FB60F9297
:1039B00011242F938F939F93EF93FF93E0914203F2
:1039C000F09143038081E0914803F091490382FD27
:1039D00012C0908180914B038F5F8F7320914C03B5
:1039E000821751F0E0914B03F0E0EE5CFC4F958FB5
:1039F00080934B0301C08081FF91EF919F918F9144
:103A00002F910F900FBE0F901F901895FC01809181
:103A1000F304811103C08FEF9FEF08959FB7F894CF
:103A200082E08093E9002091F20030E01216130644
:103A300014F421E030E02115310559F0289884E68E
:103A40008093F2048091F10080838091F2008823BA
:103A500019F09FBFC90108958BE68093E800F9CF64
:103A60002FB7F89483E08093E9009091E800892FC4
:103A7000807295FF04C09091F20080E4891B2FBFF3
:103A800008958091F80481110DC082E08093F404C0
:103A900084E08093F5041092F7041092F60481E01C
:103AA0008093F80484EF94E00895CF92DF92EF9230
:103AB000FF920F931F93E82FF92F05C001501109B2
:103AC0002109310961F1908196239417B9F305C05A
:103AD000015011092109310911F1908196239413A4
:103AE000F7CFC12CD12CE12CF12C0AC08FEFC81AD2
:103AF000D80AE80AF80A0C151D052E053F0579F0CD
:103B000080818623841791F36C2D7D2D8E2D9F2D22
:103B10001F910F91FF90EF90DF90CF90089560E09C
:103B200070E080E090E01F910F91FF90EF90DF90A8
:103B3000CF90089584EA91E09093CE048093CD04D1
:103B40008091D7049091D804009711F00E94452AE3
:103B50008091D1049091D204009711F00E94452ADF
:103B60008091D5049091D604009711F00E94452AC7
:103B70008091CF049091D004009711F00E94452AC3
:103B80008091D3049091D404009711F00C94452AAD
:103B90000895CF93DF93CDB7DEB7CB56D1090FB6DB
:103BA000F894DEBF0FBECDBF789484B5826084BD2B
:103BB00084B5816084BD85B5826085BD85B5816031
:103BC00085BD80916E00816080936E0010928100AF
:103BD000809181008260809381008091810081606A
:103BE000809381008091800081608093800080912B
:103BF0009100826080939100809191008160809318
:103C00009100809190008160809390008091C1002C
:103C100084608093C1008091C10082608093C10064
:103C20008091C10081608093C1008091C300816058
:103C30008093C3008091C00082608093C000809117
:103C4000C20081608093C20080917A00846080937A
:103C50007A0080917A00826080937A0080917A0065
:103C6000816080937A0080917A00806880937A00E6
:103C70001092F30410927A02109279028091D70088
:103C800081608093D70080EA8093D80089B58061F5
:103C900089BD89B5826089BD09B400FEFDCF61E0B0
:103CA00070E080E090E00E94CC0E8091D8008F7C84
:103CB00080618093D8008091E000807F8093E00055
:103CC0008091E1008E7E8093E1008DE08093E200A0
:103CD000559A209AEEEFFFE7859194918B3F9C4D8A
:103CE00019F481E080937802E0914203F09143035C
:103CF00082E08083E0913E03F0913F031082E091E7
:103D00004003F09141038FEC808310924A03E091CD
:103D10004603F091470386E08083E0914403F091ED
:103D20004503808180618083E0914403F0914503E5
:103D3000808188608083E0914403F0914503808115
:103D400080688083E0914403F091450380818F7DFA
:103D500080838AE090E0A0E0B0E080933603909307
:103D60003703A0933803B093390382E393E00E94B2
:103D7000A40C892B21F088EC91E00E94761582E357
:103D800093E00E94A40C1816190624F482E393E031
:103D90000E942E1980E090E00E9413181092C70232
:103DA0001092C602109210031092310310920E036B
:103DB00081E080930D031092E80261E082E00E94AE
:103DC0000D0E61E083E00E940D0E8091B9008E7FA0
:103DD0008093B9008091B9008D7F8093B90088E409
:103DE0008093B80085E48093BC0064EF71E080E0CC
:103DF00090E00E94CC0E8BE08093E20469E070E0DA
:103E00008091DF049091E0040E94DD2AFC0100977C
:103E100069F09093E0048093DF0483E08093E104F1
:103E200084E1808386E1838384E0868381E00E944D
:103E3000B80982E1898385E18A838CE08B831092C3
:103E4000D0041092CF041092D2041092D104109298
:103E5000D4041092D3041092D6041092D504109278
:103E6000DE041092DD0483E08093D9048091D704AE
:103E70009091D804892B11F080E00BC083E090E092
:103E80000E94B0299093D8048093D704892BA1F77E
:103E900019C09091D904891790F4282F30E0E0914F
:103EA000D704F091D804E20FF31FA1E0B0E0AC0F0B
:103EB000BD1FA20FB31F9C9190838F5FEACF8BE051
:103EC0008093DA0480ED97E09093DC048093DB0428
:103ED00031EEA2963FAFA297412C512C3201812C9A
:103EE000912C5401C12CD12C7601A2964FADA297F2
:103EF0004C3328F46CE97FEF88E690E004C064E678
:103F000070E088E99FEF0E94931261E08BE792E0F6
:103F10000E94731780917B0290917C02C80ED91E7B
:103F2000E11CF11C80917D0290917E02880E991E09
:103F3000A11CB11C80917F0290918002480E591EF5
:103F4000611C711C8091D1049091D204892B39F0AD
:103F50008091CF049091D004892BD1F41CC00091A2
:103F6000D90410E0C801880F991F0E94B0299093CE
:103F7000D2048093D104009709F4C3C0FC0180E00F
:103F800090E08017910724F7119211920196F9CFD2
:103F900000E010E01DC00091D90410E0C801880FB6
:103FA000991F0E94B0299093D0048093CF0400976A
:103FB00009F4A7C02091DB043091DC04FC0180E00F
:103FC00090E08017910724F7219331930196F9CF60
:103FD00061E0CE018F5B9F4F0E9473178091D904DF
:103FE000A82FB0E0A696BFAFAEAFA697FE01319660
:103FF0001F01E05CFF4F9E012F5D3F4FA4963FAF36
:104000002EAFA497A901AC963FAE2EAEAC9760E060
:1040100070E0A6968EAD9FADA69768177907BCF5A0
:1040200001151105A1F0DA012D913C91808191815A
:104030002817390760F0AC96AEADBFADAC972D91A7
:104040003C91808191818217930748F010C0808154
:104050009181DA018D939C930115110561F780819F
:104060009181AC96AEADBFADAC978D939C936F5FD5
:104070007F4FAC962EAD3FADAC972E5F3F4FAC96C9
:104080003FAF2EAFAC9732964E5F5F4FC2CF0F5F00
:104090001F4F0A30110509F09BCF6091CF0470913A
:1040A000D004A091D104B091D20480E090E020919E
:1040B000D90430E08217930724F5F1012191319161
:1040C0001F014D915C9111974217530718F41196F7
:1040D0003C932E93A496EEADFFADA4972191319120
:1040E000A496FFAFEEAFA497FB0140815181241746
:1040F000350710F43183208301966E5F7F4F12964F
:10410000D6CFA2962FADA2972F5FA2962FAFA297E0
:10411000293509F0EACE60E070E080E090E00E948E
:104120009312C701B60128E730E040E050E00E945A
:10413000872730937C0220937B02C501B40128E7D6
:1041400030E040E050E00E94872730937E022093C9
:104150007D02C301B20128E730E040E050E00E9458
:1041600087273093800220937F0280E00E94B80965
:1041700081E00E94B8090E9489150E948915811169
:104180000DC02898209A88EE91E00E94761568E884
:1041900073E180E090E00E94CC0EF5CF6FEF80E2FB
:1041A0000E94591560E283E20E94591560E084E2A2
:1041B0000E94591500E014E0C12CD12C76018091A9
:1041C0008F040E94411467E28FE194E00E94FF0295
:1041D0000E94E41380938C0461E080918F040E941C
:1041E0004B148FE194E00E94B3020E94E4130E94FA
:1041F000E21480918A0490918B04092E000CAA0B82
:10420000BB0BC80ED91EEA1EFB1E01501109B9F6E0
:10421000C701B60120E034E040E050E00E941E27D4
:1042200030938402209383020E94A70E709382022F
:104230006093810280E00E94B80981E00E94B80981
:104240000E9492160E94921681110DC02898209A01
:1042500084E092E00E94761568E873E180E090E0E7
:104260000E94CC0EF5CF8091AC049091AD048330C8
:104270009105A9F460E081E20E94851667E580E27D
:104280000E94851664E684E20E94851660E285E25B
:104290000E94851660E086E20E9485161CC0029787
:1042A00031F468E083E20E94681667E405C060E0CC
:1042B00083E20E94681667E280E20E9468166CE062
:1042C00080E00E944B1660E281E00E944B1660E0A5
:1042D00082E00E944B1600E014E060E070E0CB0149
:1042E000A7966FAFA797A8967FAFA897A9968FAF0D
:1042F000A997AA969FAFAA970E94D215C09093043F
:10430000D09094040D2C000CEE08FF08A7966FAD1A
:10431000A797A8967FADA897A9968FADA997AA96BB
:104320009FADAA976C0D7D1D8E1D9F1D015011091B
:10433000B9F620E034E040E050E00E941E273093C0
:1043400086022093850280E00E94B8095D98559A04
:10435000E091C104F091C2040190F081E02D81EC64
:1043600094E009958823A1F36AE070E080E090E092
:104370000E94CC0EE091C104F091C2040190F08142
:10438000E02D81EC94E00995882311F3E091C104BC
:10439000F091C2040190F081E02D81EC94E0099548
:1043A0008111F4CF6AE070E080E090E00E94CC0ED2
:1043B000E091C104F091C2040190F081E02D81EC04
:1043C00094E009958111E2CF0E94251061157105D5
:1043D0008105910511F00E94C42664EF71E080E030
:1043E00090E00E94CC0E0E9425107093960260937C
:1043F0009502FF24F3948EE8C82E83E0D82E812CFA
:10440000912C90E8A92E9FE3B92E23E3422E542C41
:1044100023EB622E2FE3722E5D9A559A80E00E9464
:10442000B809289A209A0E940E088091A80281114A
:1044300004C0F092A8020E942713F89420918702EA
:1044400030918802109288021092870278948091AD
:10445000AD029091AE02820F931F9093AE028093B3
:10446000AD02B6010E9490287093AA026093A9023F
:104470008091A802811104C0F092A8020E94271323
:10448000F8942091890230918A0210928A02109247
:10449000890278948091AF029091B002820F931FAD
:1044A0009093B0028093AF02B6010E94902870935F
:1044B000AC026093AB020E943A070E945C060E9425
:1044C000AF070E94AB090E94251020919502309100
:1044D00096028B01021B130B1093B2020093B102E0
:1044E00082E393E00E94A40C1816190644F482E3B8
:1044F00093E00E942E199093B5028093B4028091AC
:10450000B4029091B5028133910519F4F092B3028F
:1045100004C0C09711F41092B3028091B3028823B3
:1045200009F446C040920A0150920B0160920C01BE
:1045300070920D018091A402863041F08091A50215
:10454000863059F48091A602863039F460E070E03C
:1045500080E090E00E949312ACC28091A302882375
:1045600079F0013D174060F08091A1029091A20284
:1045700097FF03C09195819591098D3A9D4034F73D
:1045800080919B0290919C02853F9140FCF6809126
:104590009F029091A002853F9140C4F680919D02B8
:1045A00090919E02853691058CF60E94BF0981C2CA
:1045B00080920A0190920B01A0920C01B0920D0121
:1045C0008091A302882309F48CC0013D174008F4B0
:1045D00088C08091A1029091A20297FF03C091959B
:1045E000819591098D3A9D400CF47BC081E090E06B
:1045F0000E9413182898209A60E070E080E090E014
:104600000E94931268EE73E080E090E00E94CC0E6E
:104610008091A502811129C00E940E080E94AF0757
:104620006EEC7FEF8CEC9FEF0E94931280919B02C7
:1046300090919C02873991054CF00E94251070934F
:104640009A02609399020E94AB0933C080919D0247
:1046500090919E028536910584F780919F029091FA
:10466000A00289379105A4F2E8CF8091A6028823A1
:1046700099F2E3CF0E94AB090E94AF076EEC7FEF87
:104680008CEC9FEF0E94931280919B0290919C0270
:1046900087399105ACF480919D0290919E028536F8
:1046A000910574F480919F029091A0028937910541
:1046B0003CF48091970290919802883E9340D0F20A
:1046C00060E070E080E090E00E94931210928C0213
:1046D00010928B021092A2021092A1020E945C061C
:1046E000DCC18091A502863009F074C18091A602D8
:1046F000863009F06FC181E090E00E94131881E0DC
:104700000E94B809109291021092920210929302A4
:104710001092940210928D0210928E0210928F02CB
:10472000109290020E943A0780918D0290918E0221
:10473000A0918F02B09190024497A105B1055CF45D
:104740000E943A070E94AF0764E670E08AE190E0B9
:104750000E949312E9CF0E943A0780918D029091B6
:104760008E02A0918F02B09190028D97A105B105A4
:104770009CF40E943A070E94AF0764E670E08AE169
:1047800090E00E94931280919F029091A00289571D
:1047900091098B37914008F70E94AF0780919F02E3
:1047A0009091A002883791054CF40E94AF0764E60F
:1047B00070E088E690E00E949312F0CF0E943A07E2
:1047C00080918D0290918E02A0918F02B091900203
:1047D0000B97A105B1051CF10E943A070E94AF0793
:1047E00080919B0290919C02875991098D3591404F
:1047F00018F460E070E00EC080919F029091A002DA
:10480000895791098B37914018F464E670E002C033
:1048100069E170E088E690E00E949312D1CF64E6EF
:1048200070E088E690E00E9493120E940E080E94B9
:10483000251070939A02609399028091A7028630A6
:1048400078F40E940E080E94AF070E94BF090E94E0
:10485000AB098091970290919802893B9B4068F345
:104860000E940E088091A702863039F40E940E083B
:104870000E94AF070E94BF09F5CF0E9425107093D8
:104880009A02609399020E94AB09809197029091DD
:104890009802883B9B4028F40E94AF070E94BF0902
:1048A000F2CF109291021092920210929302109203
:1048B000940210928D0210928E0210928F0210922A
:1048C00090020E943A0780918D0290918E02A091F1
:1048D0008F02B09190028D3E9F4FAF4FBF4F5CF063
:1048E0000E943A070E94AF0769E170E088E690E015
:1048F0000E949312E8CF0E943A0780918D02909116
:104900008E02A0918F02B0919002843D9F4FAF4FD5
:10491000BF4F9CF00E943A070E94AF0769E170E028
:1049200088E690E00E94931280919B0290919C02F5
:10493000875991098D35914000F70E94AF0780910A
:104940009B0290919C02863991054CF40E94AF071E
:1049500064E670E088E690E00E949312F0CF0E9437
:104960003A0780918D0290918E02A0918F02B091B2
:104970009002863F9F4FAF4FBF4F2CF50E943A07E2
:104980000E94AF0780919F029091A00289579109E0
:104990008B37914028F464E670E080E090E010C02E
:1049A00080919B0290919C028759910964E670E086
:1049B0008D35914018F488E690E002C08AE190E0DD
:1049C0000E949312CECF64E670E088E690E00E94E9
:1049D000931263C080919B0290919C028134F6E017
:1049E0009F0744F020919F023091A002213436406D
:1049F0000CF0ACCD9C01255F314080919D029091DF
:104A00009E022B34344048F49C012D523140233F08
:104A1000314018F40E949A0A4CC020919F023091B4
:104A2000A002255F31402B34344030F49C012D52DC
:104A30003140233F314070F385569109873C910501
:104A400008F0B3CD2898209A81E090E00E941318D6
:104A50000E94251070939A026093990280919B02A4
:104A600090919C0286399105C4F480919F029091A7
:104A7000A002883791058CF40E94AB090E94AF0711
:104A80006CE97FEF88E99FEF0E9493128091970273
:104A900090919802893B9B4008F31092A3020E94D8
:104AA0002510709396026093950280E090E00E943A
:104AB00013180E94B00CB0CCE2E3F3E01382128230
:104AC00088EE93E0A0E0B0E084839583A683B7836B
:104AD00022E631E0318320832DEC30E035872487D6
:104AE0002CEC30E03787268728EC30E0318B208BA8
:104AF00029EC30E0338B228B2AEC30E0358B248B91
:104B00002EEC30E0378B268B118E128E138E148E86
:104B1000EFECF3E01382128284839583A683B7833C
:104B200024E731E0318320832FEF3FEF358724875F
:104B3000EFE1F4E01382128284839583A683B78326
:104B400086E891E091838083EFEDF4E0118210829A
:104B500012828FEF838315821482168285EA91E098
:104B60009287818782E492E09487838784EA91E048
:104B700090878783EDECF4E0138212821582148211
:104B80001782168211861086138612868AEA91E0B1
:104B900091838083E1ECF4E01282158210868EE02E
:104BA000818781E08287838788E991E09183808390
:104BB00086E0E2E5F1E0A5EAB4E001900D928A9585
:104BC000E1F786E0E8E5F1E0AFE9B4E001900D92AD
:104BD0008A95E1F7E3E9F4E084E090E0928F818F39
:104BE00014A613A615A6E6E8F4E083E090E090870B
:104BF000878313861286148640E050E063E070E0FD
:104C000089E794E00E94301240E050E063E070E0F9
:104C10008CE694E00E94301240E050E063E070E0E7
:104C20008FE594E00E94301240E050E065E070E0D3
:104C300082E594E00E94301240E050E065E070E0D0
:104C400085E494E00E94301240E050E065E070E0BE
:104C500088E394E00E94301240E050E065E070E0AC
:104C60008BE294E00C943012CF92DF92EF92FF929D
:104C70000F931F93CF93DF931F92CDB7DEB7182FFB
:104C8000062FE42E862F880F8E5F99830E9492183C
:104C900083E00E949218F12EC12E9981D92E8C2D7D
:104CA0008F19801798F4F601E7FE02C0849101C0C5
:104CB00080810E949218182F80E00E949218812310
:104CC000FFEFCF1ADF0A8111EACF01C081E00F9018
:104CD000DF91CF911F910F91FF90EF90DF90CF90D8
:104CE00008958F929F92AF92BF92CF92DF92EF92F0
:104CF000FF92CF93DF93EC01688179818A819B8158
:104D0000611571058105910521F464E279ED8BE56A
:104D100097E02DE133EF41E050E00E941E2749016A
:104D20005A019B01AC01A7EAB1E40E943D276B0147
:104D30007C01ACEEB4EFA50194010E944B27DC018D
:104D4000CB018C0D9D1DAE1DBF1DB7FF03C001978C
:104D5000A109B04888839983AA83BB83BC01CD0194
:104D60009F77DF91CF91FF90EF90DF90CF90BF9032
:104D7000AF909F908F9008950E947126089584E2CD
:104D800091E00E947126089560932401709325019B
:104D90008093260190932701089597F99F6780E8F3
:104DA00070E060E008959FEF80EC089500240A947D
:104DB0001616170618060906089500240A941216F6
:104DC0001306140605060895092E0394000C11F429
:104DD000882352F0BB0F40F4BF2B11F460FF04C0D6
:104DE0006F5F7F4F8F4F9F4F089557FD9058440F2F
:104DF000551F59F05F3F71F04795880F97FB991F3A
:104E000061F09F3F79F087950895121613061406F6
:104E1000551FF2CF4695F1DF08C016161706180683
:104E2000991FF1CF86957105610508940895E8945E
:104E3000BB2766277727CB0197F90895052E97FBA7
:104E40001EF400940E94352757FD07D00E94872743
:104E500007FC03D04EF40C943527509540953095BF
:104E600021953F4F4F4F5F4F0895909580957095D6
:104E700061957F4F8F4F9F4F08950E94A927A59F4F
:104E8000900DB49F900DA49F800D911D1124089545
:104E9000B7FF0C943D270E943D27821B930B08957A
:104EA0002F923F924F925F926F927F928F929F923A
:104EB000AF92BF92CF92DF92EF92FF920F931F9328
:104EC000CF93DF93CDB7DEB7CA1BDB0B0FB6F894D9
:104ED000DEBF0FBECDBF09942A88398848885F8419
:104EE0006E847D848C849B84AA84B984C884DF808A
:104EF000EE80FD800C811B81AA81B981CE0FD11D6E
:104F00000FB6F894DEBF0FBECDBFED010895A1E24C
:104F10001A2EAA1BBB1BFD010DC0AA1FBB1FEE1F33
:104F2000FF1FA217B307E407F50720F0A21BB30B7E
:104F3000E40BF50B661F771F881F991F1A9469F7FA
:104F400060957095809590959B01AC01BD01CF0156
:104F50000895A29FB001B39FC001A39F700D811D52
:104F60001124911DB29F700D811D1124911D089572
:104F70000E94CC270C94E4260E94DD2658F00E9463
:104F8000D62640F029F45F3F29F00C94CD2651112C
:104F90000C9418270C94D3260E94F52668F39923C5
:104FA000B1F3552391F3951B550BBB27AA27621725
:104FB0007307840738F09F5F5F4F220F331F441F32
:104FC000AA1FA9F335D00E2E3AF0E0E832D0915066
:104FD0005040E695001CCAF72BD0FE2F29D0660F53
:104FE000771F881FBB1F261737074807AB07B0E896
:104FF00009F0BB0B802DBF01FF2793585F4F3AF09C
:105000009E3F510578F00C94CD260C9418275F3FF5
:10501000E4F3983ED4F3869577956795B795F79521
:105020009F5FC9F7880F911D9695879597F9089509
:10503000E1E0660F771F881FBB1F621773078407A5
:10504000BA0720F0621B730B840BBA0BEE1F88F7B4
:10505000E09508950E9431286894B1110C941827A6
:1050600008950E94FD2688F09F5798F0B92F992740
:10507000B751B0F0E1F0660F771F881F991F1AF043
:10508000BA95C9F714C0B13091F00E941727B1E06A
:1050900008950C941727672F782F8827B85F39F069
:1050A000B93FCCF3869577956795B395D9F73EF4DC
:1050B00090958095709561957F4F8F4F9F4F089584
:1050C000DB018F939F930E943D27BF91AF91A29FD9
:1050D000800D911DA39F900DB29F900D11240895F6
:1050E000991B79E004C0991F961708F0961B881F3A
:1050F0007A95C9F780950895AA1BBB1B51E107C09B
:10510000AA1FBB1FA617B70710F0A61BB70B881F57
:10511000991F5A95A9F780959095BC01CD010895E6
:1051200097FB072E16F4009407D077FD09D00E9454
:105130007C2807FC05D03EF4909581959F4F0895FB
:10514000709561957F4F0895EE0FFF1F0590F491C4
:10515000E02D09940E94A927B7FF0895821B930BA5
:10516000089597FB57FF0C94C1289F938F930E943B
:10517000C1286E1B7F0BAF91BF918A0B9B0B0895CB
:10518000E894DF93CF93FC01DB010E94A9277F9372
:105190006F93E9019A01AC01BF93AF933F932F93B3
:1051A000DF010E94A92726F46C1B7D0B820B930B59
:1051B0009E01EB01FC010E948B29AF91BF912F91C1
:1051C0003F910E948B29BE01CF01F9012F913F91A0
:1051D000CF91DF910895689401C0E894F92FF12BE5
:1051E00012F00C941F29A0E0B0E0E9EFF8E20C9473
:1051F0005627092E059422F40E947B29112392F44C
:10520000F0E80F26FFEFE094F09400951095B0942D
:10521000C094D094A194BF0ACF0ADF0AEF0AFF0A14
:105220000F0B1F0B0E942A2907FC0E947B29CDB778
:10523000DEB7ECE00C947227689401C0E8948F927A
:105240009F92CF93DF930E942A29DF91CF919F9065
:105250008F90089588249924F401E401B0E49F9389
:10526000AA279A158B049C04ED05FE05CF05D007EF
:10527000A10798F4AD2FDC2FCF2FFE2FE92D982C0E
:10528000892E982F872F762F652F542F432F322F5B
:105290002227B85031F7BF9127C01B2EBF91BB27E3
:1052A000220F331F441F551F661F771F881F991F2A
:1052B000881C991CEE1FFF1FCC1FDD1FAA1FBB1FE0
:1052C0008A149B04EC05FD05CE05DF05A007B10798
:1052D00048F08A189B08EC09FD09CE09DF09A00BEC
:1052E000B10B21601A94E1F62EF49401AF01BE01D6
:1052F000CD01000C0895609570958095909530953E
:105300004095509521953F4F4F4F5F4F6F4F7F4FC7
:105310008F4F9F4F08950E94A927460F571FC81F00
:10532000D91F08F4319608950F931F93CF93DF93FD
:10533000869F8001879F100D969F100D1124C80134
:105340000E94B029EC01009729F0A80160E070E00C
:105350000E94B52BCE01DF91CF911F910F9108953F
:10536000CF93DF938230910510F482E090E0E091DA
:105370000205F091030520E030E0C0E0D0E0309776
:1053800011F14081518148175907C0F0481759075A
:1053900061F482819381209719F09B838A832BC0CB
:1053A000909303058093020526C02115310519F05D
:1053B0004217530718F49A01BE01DF01EF01028082
:1053C000F381E02DDCCF2115310509F1281B390BC4
:1053D0002430310590F412968D919C9113976115AC
:1053E000710521F0FB019383828304C09093030530
:1053F00080930205FD01329644C0FD01E20FF31FC8
:1054000081939193225031092D933C933AC020917E
:10541000000530910105232B41F420912A013091A0
:105420002B01309301052093000520912801309134
:1054300029012115310541F42DB73EB740912C01CA
:1054400050912D01241B350BE0910005F0910105D1
:10545000E217F307A0F42E1B3F0B2817390778F04B
:10546000AC014E5F5F4F2417350748F04E0F5F1FAA
:1054700050930105409300058193919302C0E0E0B1
:10548000F0E0CF01DF91CF9108950F931F93CF9359
:10549000DF93009709F48CC0FC01329713821282CB
:1054A00000910205109103050115110581F4208179
:1054B0003181820F931F209100053091010528173B
:1054C000390779F5F0930105E093000571C0D80123
:1054D00040E050E0AE17BF0750F412962D913C917A
:1054E0001397AD012115310509F1D901F3CF9D01C4
:1054F000DA013383228360817181860F971F8217BF
:10550000930769F4EC0128813981260F371F2E5F3C
:105510003F4F318320838A819B8193838283452BF4
:1055200029F4F0930305E093020542C01396FC931F
:10553000EE931297ED01499159919E01240F351F69
:10554000E217F30771F480819181840F951F029611
:1055500011969C938E938281938113969C938E9344
:105560001297E0E0F0E0D80112968D919C9113978C
:10557000009719F0F8018C01F6CF8D919C9198015C
:105580002E5F3F4F820F931F209100053091010540
:105590002817390769F4309729F4109203051092FF
:1055A000020502C0138212821093010500930005C8
:1055B000DF91CF911F910F910895A0E0B0E0E3EE4D
:1055C000FAE20C945427EC01009721F4CB010E94DD
:1055D000B029B8C0FC01E60FF71F9C012250310929
:1055E000E217F30708F4ACC0D9010D911C91119793
:1055F00006171707B0F00530110508F49FC0C80161
:1056000004978617970708F499C002501109061BE2
:10561000170B019311936D937C93CF010E94452A40
:105620008DC05B01A01AB10A4C01800E911EA091A1
:105630000205B091030540E050E0E12CF12C1097F9
:1056400009F44AC0A815B905D1F56D907C90119761
:10565000630182E0C80ED11CCA14DB0480F1A301EF
:105660004A195B096A0182E0C80ED11C1296BC90EF
:1056700012971396AC91B5E0CB16D10440F0B282EC
:10568000A38351834083D9016D937C930AC00E5F3D
:105690001F4FC301800F911FF90191838083EB2D70
:1056A000FA2FE114F10431F0D7011396FC93EE9335
:1056B000129744C0F0930305E09302053FC08D911B
:1056C0009C9111974817590708F4AC017D01129677
:1056D0000D90BC91A02DB3CF809100059091010554
:1056E00088159905E1F446175707C8F480912801F9
:1056F00090912901009741F48DB79EB740912C01FC
:1057000050912D01841B950BE817F907C8F4F0930D
:105710000105E0930005F901718360830FC0CB019F
:105720000E94B0297C01009759F0A801BE010E9497
:10573000AC2BCE010E94452AC70104C0CE0102C095
:1057400080E090E0CDB7DEB7EEE00C94702781E00A
:1057500090E0F8940C94BC2BFB01DC0102C001909A
:105760000D9241505040D8F70895DC0101C06D936F
:1057700041505040E0F7089510E0C4EED0E004C07E
:10578000FE010E94A4282196C53ED107C9F7F894CE
:02579000FFCF49
:105792000F00F401D007040004010000803F320D25
:1057A200320D320D320D320DFFFFFFFF00E100001E
:1057B2000000000001000000000004058000040059
:1057C2000F0020003700550078009C01B501CF0181
:1057D200EA0107022602470269028E02B502DE02D0
:1057E2000A03018001800180FF7FFF7FFF7F0000AD
:1057F20000008E19F4181F19D519A40C2E1942197C
:1058020000000000BA0C060F7D0DD00CDB0C810DE0
:105812009F0D00000000FF02CF022F03A302C70268
:10582200B302A40200000000790E000000008B0FFA
:10583200000000005019000000008B0F00C18081A1
:105842000000004672656D646D657373756E672046
:1058520065726B616E6E7400426C7565746F6F7405
:105862006876657262696E64756E672068657267D4
:10587200657374656C6C74004665686C657220446F
:105882007265686265776567756E677373656E7357
:105892006F7273004665686C657220426573636857
:1058A2006C65756E6967756E677373656E736F721B
:0658B20073000D0A000066
:2070000055C000006EC000006CC000006AC0000068C0000066C0000064C0000062C0000043
:2070200060C000005EC00000F2C400005AC0000058C0000056C0000054C0000052C00000EE
:2070400050C0000078C000004CC000004AC0000048C0000046C0000044C0000042C00000BE
:2070600040C000003EC000003CC000003AC0000038C0000036C0000034C0000032C0000048
:2070800030C000002EC000002CC000002AC0000028C0000026C0000024C0000022C00000A8
:2070A00020C000001EC000001CC0000011241FBECFEFDAE0DEBFCDBF11E0A0E0B1E0E2E3BC
:2070C000FFE702C005900D92A83AB107D9F711E0A8EAB1E001C01D92AE3BB107E1F78FD30B
:2070E00026C78ECFF89410926F0010928100109285001092840081E085BF15BE47985D9AEB
:20710000289A0C94000008952091B2013091B3012F5F3F4F3093B3012093B201932F37FFA6
:2071200003C08EEF831B982F990F921710F447980895479A08951F920F920FB60F9211246E
:207140002F938F939F93EF93FF9310928500109284008091A8019091A901009741F00197D3
:207160009093A9018093A801892B09F45D9A8091AA019091AB01009741F001979093AB0126
:207180008093AA01892B09F4289AE0E0F0E0859194918F5F9F4F49F08091AC019091AD0151
:2071A00001969093AD018093AC01FF91EF919F918F912F910F900FBE0F901F90189584E0BC
:2071C0008093E9000DC08091E8008B778093E80003C08EB3882351F08091E80082FFF9CFBE
:2071E0008091E80085FFEFCF8091F1000895982F83E08093E9008091E80085FD0DC0809136
:20720000E8008E778093E80003C08EB3882369F08091E80080FFF9CF9093F1005D9884E6CB
:2072200090E09093A9018093A80108954F925F926F927F928F929F92AF92BF92CF92DF921E
:20724000EF92FF920F931F93CF93DF9384E08093E9008091E80082FF57C2289884E690E067
:207260009093AB018093AA01AADF182F853481F48CE49DE19093AD018093AC0107B600FC4B
:20728000FDCFF999FECF81E180935700E89503C0843519F494DF8DE00DC28C34E1F38035F9
:2072A000D1F3843721F484E4A2DF80E003C2813611F489E5FFC18134B1F481DF182F7FDFE3
:2072C00090E0880F991FAA2797FDA095BA2F312F330F20E0442737FD4095542F822B932B68
:2072E000A42BB52BB8C1803711F483E5E3C1833549F4C0E0D1E089917ADF21E0C730D20714
:20730000D1F7D9C1863521F481E371DF80E3D2C1833731F487E86BDF85E969DF8EE1CAC149
:207320008536B9F4E0E0F0E093E085E090935700E89507B600FCFDCF80935700E89507B65D
:2073400000FCFDCFE058FF4FA0E7E030FA0771F7A2CF823739F4E1E0F0E089E08093570024
:207360008491A8C1863439F4E0E0F0E089E08093570084919FC18E3439F4E3E0F0E089E0E5
:2073800080935700849196C1813539F4E2E0F0E089E08093570084918DC1823631F489E521
:2073A00026DF80E024DF80E885C1823419F0873609F0E5C01092AD011092AC0100DF082FE8
:2073C000FEDEF82EFCDE682E8554823008F071C1902F80E0CF2DD0E0C82BD92B10926F00B3
:2073E000173609F04BC081E180935700E895DD24CC24C3943FC0E090AE01F090AF010091CC
:20740000B0011091B101B6E46B16D9F4ED2DF0E0EE29FF29E4918E2FEADEDD2081F082E08D
:2074200090E0A0E0B0E0E80EF91E0A1F1B1FE092AE01F092AF010093B0011093B101DC2470
:2074400018C0D801C701B695A7959795879559D5CEDE82E090E0A0E0B0E0E80EF91E0A1FF2
:207460001B1FE092AE01F092AF010093B0011093B1012197209709F0BECF7DC08090AE01F5
:207480009090AF01A090B001B090B10196E4691609F05DC083E0F40180935700E89507B63E
:2074A00000FCFDCF54C0F6E46F1661F5772031F1E090AE01F090AF010091B0011091B1019E
:2074C0007EDED82ECC24852D90E08C299D29F7010C0140925700E895112482E090E0A0E08B
:2074E000B0E0E80EF91E0A1F1B1FE092AE01F092AF010093B0011093B10102C060DE582E1A
:20750000742423C0E090AE01F090AF010091B0011091B10116950795F794E79450DE682FFA
:20752000C701F7D48091AE019091AF01A091B001B091B1010296A11DB11D8093AE01909349
:20754000AF01A093B001B093B101219704C05524772444244394209709F0A5CF96E46916B6
:2075600041F485E0F40180935700E89507B600FCFDCF8DE03CDE82E080936F009CC0833492
:2075800071F40091AE011091AF0119DE90E021E0F8010C0120935700E89511247CCE8336C8
:2075A00019F5E090AE01F090AF010091B0011091B10105DEF701E16090E021E00C0120938C
:2075C0005700E895112482E090E0A0E0B0E0E80EF91E0A1F1B1FE092AE01F092AF0100936A
:2075E000B0011093B10157CE8D3661F4E091AE01F091AF0185E080935700E89507B600FCF2
:20760000FDCF49CE823551F4E091AE01F091AF0105911491812FEBDD802F4CC0843421F5FE
:20762000E090AE01F090AF010091B0011091B10116950795F794E794C2DD682FC70169D4DE
:207640008091AE019091AF01A091B001B091B1010296A11DB11D8093AE019093AF01A093D8
:20766000B001B093B10117CE843609F5E090AE01F090AF010091B0011091B101D801C70142
:20768000B695A795979587953CD4B1DD82E090E0A0E0B0E0E80EF91E0A1F1B1FE092AE010A
:2076A000F092AF010093B0011093B10104C08B3111F08FE39CDD83E08093E9009091E8002B
:2076C0008091E8008E778093E80095FF04C010C08EB38823C9F08091E80080FFF9CF809193
:2076E000E8008E778093E80003C08EB3882361F08091E80080FFF9CF84E08093E9008091F1
:20770000E8008B778093E800DF91CF911F910F91FF90EF90DF90CF90BF90AF909F908F90AC
:207720007F906F905F904F9008959091B601892F8F77813249F58091B7018032A1F081328A
:2077400019F5913A09F58091E800877F8093E8008DE091E067E070E00BD28091E8008B770B
:207760008093E8000895913279F48091E800877F8093E8008DE091E067E070E05DD2809192
:20778000E8008E778093E800089582E061EC42E0B5D083E061E842E1B1D084E060E842E1EF
:2077A000ADC084B7877F84BF88E10FB6F89480936000109260000FBE20E880E090E00FB63F
:2077C000F89420936100809361000FBE81E085BF92E095BF3F9A209A559AE1E6F0E02083A1
:2077E000108247985D9A289A109289008AEF8093880090936F0083E080938100F0C0409116
:20780000000850910108109201081092000894B714BE88E10FB6F8948093600010926000D5
:207820000FBE292F30E0F901E270F07091FD18C090FF05C0859194918F5F9F4F81F423FFFF
:207840000FC08091090190910A014817590741F0E0E0F0E0859194918F5F9F4F09F042DC64
:20786000A0DF78941092AD011092AC010CC0DEDC36D38091AC019091AD0181549F4110F00D
:207880001092140141DC80911401882381F78091E00081608093E00025DC80E090E0089598
:2078A000FA01923049F0933061F09130F9F485E191E022E130E01EC087E291E02EE330E04D
:2078C00019C0882329F485E691E024E030E012C0813029F489E691E022E230E00BC0823006
:2078E00029F48DE891E028E130E004C080E090E020E030E091838083C90108958093E9004E
:207900008091EB0081608093EB001092ED006093EC004093ED008091EE00881F8827881F62
:2079200008958091B60188238CF403C08EB38823B1F08091E80082FFF9CF8091E8008B772A
:207940008093E80008958EB3882349F08091E80080FFF9CF8091E8008E778093E800089594
:20796000EF92FF920F931F9345D04CD008ED10E0F80180818F77808380818068808380819B
:207980008F7D808319BC1EBA1092B40180EEE82EF12CF70180818B7F8083F8018081816052
:2079A000808380E060E042E0A9DFE1EEF0E080818E7F8083E2EEF0E0808181608083808144
:2079C00088608083F70180818E7F8083F8018081806180831F910F91FF90EF900895E7ED06
:2079E000F0E08081816080838AE482BF81E08093B501B6CFE8EDF0E080818E7F808310921C
:207A0000E20008951092DA001092E10008951F920F920FB60F9211242F933F934F935F93F6
:207A20006F937F938F939F93AF93BF93EF93FF938091DA0080FF1BC08091D80080FF17C0B2
:207A40008091DA008E7F8093DA008091D90080FF0BC080E189BD82E189BD09B400FEFDCF36
:207A600081E08EBB3BD203C019BC1EBA37D28091E10080FF17C08091E20080FF13C0809138
:207A8000E2008E7F8093E2008091E20080618093E2008091D80080628093D80019BC85E049
:207AA0008EBB1CD28091E10084FF2CC08091E20084FF28C080E189BD82E189BD09B400FEC5
:207AC000FDCF8091D8008F7D8093D8008091E1008F7E8093E1008091E2008F7E8093E20012
:207AE0008091E20081608093E2008091B401882331F48091E30087FD02C081E001C084E067
:207B00008EBBECD18091E10083FF21C08091E20083FF1DC08091E100877F8093E10082E06A
:207B20008EBB1092B4018091E1008E7F8093E1008091E2008E7F8093E2008091E2008061E9
:207B40008093E20080E060E042E0D8DEC7D1FF91EF91BF91AF919F918F917F916F915F9130
:207B60004F913F912F910F900FBE0F901F9018959C014091BC015091BD014617570718F49D
:207B8000F90190E044C06115710511F0AB01F8CF8091E8008E778093E80040E050E0F0CF0F
:207BA0008EB3882309F444C0853009F443C08091E80083FF02C081E008958091E80082FD70
:207BC00031C08091E80080FF22C08091F3009091F200782F60E0292F30E0262B372B07C07A
:207BE00081918093F100415050402F5F3F4F4115510519F02830310598F390E02830310566
:207C000009F491E08091E8008E778093E8004115510531F6992321F605C08EB3882341F075
:207C2000853041F08091E80082FFF7CF80E0089582E0089583E008959C016115710529F47C
:207C40008091E8008B778093E800F90126C08EB3882391F1853091F18091E80083FF02C06C
:207C600081E008958091E80082FFF1CF06C08091F10081936150704059F02091F300809191
:207C8000F200322F20E090E0822B932B892B79F78091E8008B778093E80061157105B9F601
:207CA00005C08EB3882341F0853041F08091E80080FFF7CF80E0089582E0089583E00895C2
:207CC0000F931F93DF93CF9300D0CDB7DEB7E6EBF1E08091F100819381E0EE3BF807C9F792
:207CE00024DD8091E80083FFE4C08091B6019091B701953009F46DC0963040F4913081F1A7
:207D0000913070F0933009F0D4C02AC0983009F4A3C0993009F4B2C0963009F0CAC07CC023
:207D2000803809F4C6C0823809F0C3C08091BA0187708093E9008091EB001092E9002091DB
:207D4000E800277F2093E80090E025E0969587952A95E1F781708093F1001092F10087C0D8
:207D6000882319F0823009F0A4C08F71823009F0A0C08091B801882331F52091BA01277097
:207D800009F497C02093E9008091EB0080FF1BC0933021F48091EB00806213C08091EB0018
:207DA00080618093EB0081E090E002C0880F991F2A95E2F78093EA001092EA008091EB00E5
:207DC00088608093EB001092E9008091E800877F51C0882309F06DC01091B8011F770FB79B
:207DE000F8948091E800877F8093E8009ADD8091E80080FFFCCF8091E3008078812B809398
:207E0000E30080688093E300112311F482E001C083E08EBB0FBF4DC08058823008F049C033
:207E20008091B8019091B9016091BA01AE014F5F5F4F36DDBC01009709F43BC08091E8008E
:207E4000877F8093E80089819A8192DE8091E8008B778093E8002DC0803859F58091E800AA
:207E6000877F8093E8008091B4018093F1008091E8008E778093E80054DD1BC08823C9F4CA
:207E80009091B8019230A8F48091E800877F8093E8009093B40145DD8091B401882331F420
:207EA0008091E30087FD02C081E001C084E08EBB6CDC8091E80083FF0AC08091EB0080624E
:207EC0008093EB008091E800877F8093E8000F900F90CF91DF911F910F91089508951F9360
:207EE0008EB3882361F01091E9001092E9008091E80083FF01C0E4DE17701093E9001F916F
:207F00000895F999FECF92BD81BDF89A992780B50895262FF999FECF1FBA92BD81BD20BDBD
:207F20000FB6F894FA9AF99A0FBE01960895F894FFCF4341544552494E4100777700080031
:207F40000000000000080112011001020000084123360001000201000109023E00020100FF
:207F600080320904000001020201000524001001042402040524060001070582030800FF0C
:207F800009040100020A000000070504021000010705830210000104030904220341007216
:207FA000006400750069006E006F0020004C0065006F006E006100720064006F0000001836
:1A7FC00003410072006400750069006E006F0020004C004C004300000000D7
:00000001FF
